:100000000C9451160C942B05189518951895189565
:100010001895189518951895189518951895189578
:100020001895189518951895189518950C945805C5
:100030000C94B0050C9448050C9460041895189520
:1000400018951895189518950C94200618951895DC
:100050000C943A06189518951895189518951895B2
:1000600018951895189518954F4B00455252003029
:1000700031323334353637383941424344454641CD
:1000800054480D0041542B51504F57443D310D0001
:10009000436F6E6E656374696E673A0041542B510D
:1000A000494F50454E3D22544350222C22002C00F3
:1000B0000D0A00222C000D0039342E3133372E3139
:1000C00039332E323138222C353135310D0041543F
:1000D0002B5153494D535441543F0D0053494D3A10
:1000E0000041542B4350494E3F0D0041542B435087
:1000F000494E3D0050494E3A0041542B435245472A
:100100003F0D0047534D3A0041542B43475245475A
:100110003F0D00475052533A0041542B434F505328
:100120003F0D0041542B51494647434E543D300D3D
:100130000041542B5149435347503D312C004F70DF
:10014000657261746F72206973204D616E75616CA8
:100150000D0A0022004F70657261746F722069731E
:10016000204D54530D0A0022696E7465726E6574D9
:100170002E6D74732E7275222C226D7473222C22B4
:100180006D747322004F70657261746F72206973B1
:10019000204D656761666F6E0D0A0022696E746599
:1001A000726E6574222C226764617461222C22674E
:1001B0006461746122004F70657261746F722069AE
:1001C00073204261696B616C57657374436F6D0D89
:1001D0000A0022696E65742E6277632E7275222C76
:1001E00022627763222C2262776322004F7065724D
:1001F00061746F7220697320556E656466696E65FF
:10020000640D0A0041542B51494D55583D300D00A5
:1002100041542B51494D4F44453D310D0041542B24
:100220005149544346473D332C322C3531322C3121
:100230000D0041542B5149444E5349503D310D005E
:1002400041542B5149444E5349503D300D004154C7
:100250002B51495245474150500D0041542B5149B3
:100260004143540D0041542B51494C4F4349500DCB
:100270000049503A004F6E2047534D0D0A0041543B
:100280005A0D0041545A3A00415445300D00415432
:1002900045303A004154483A00496E732E20534984
:1002A0004D0D0A004572722E2050494E0D0A004134
:1002B000542B434C434B3D225343222C312C2200E0
:1002C000220D0041542B434C434B3D225343222CDF
:1002D000302C220041542B435057443D225343229B
:1002E0002C2200222C22004572726F722047534D3F
:1002F0000D0A004572726F7220475052530D0A006A
:10030000496E666F206572722E00436F6E6E2E20EE
:10031000737563636573730D0A00436C6F73656473
:1003200020636F6E6E656374696F6E0D0A004E6FA9
:1003300020616E737765722066726F6D20736572CF
:100340007665720D0A004572726F7220636F6E6E71
:10035000656374696F6E20746F2073657276657261
:100360000D0A00536C6565702E002B2B2B00415439
:100370000D0041542B5149434C4F53450D00494DFD
:1003800045493D000A00434349443D004353513D24
:10039000005645523D00310030004E6F20627974A6
:1003A0006573210D0A003A30313645303030333034
:1003B000303030303030303030303038450D0A0099
:1003C0003A464636453030303333303330333033CD
:1003D000303330333037300D0A003A303136453162
:1003E0003537430D0A003A46463645313537450D17
:1003F0000A003A303136453031303039300D0A009C
:100400003A464636453031303039320D0A004E6FAB
:100410007420737570706F7274004747534D2000DD
:100420004100202843293230313100506F77657206
:100430002D55700041542B51434349440D00415404
:100440002B47534E0D0041542B4353510D000000D8
:100450000B04170001030B040D030D035203950356
:100460009E03B003B40397030B040B040B040B04AB
:100470000B040B04E203D7036F0392038E036403A0
:10048000A5030100B80B1D00C60B0E0C1C0C280C9C
:10049000310C330C390C540C5B0C6C0C6E0C720C64
:1004A0007E0C890C8D0CBC0B930CD00CD60CEC0C78
:1004B000140DBC0B240D260D280D2A0D2C0D340D0A
:1004C0003E0D0100E80B0900CB0BD00BD30BD50B75
:1004D000D80BDA0BDD0BDF0BE20B00310126116BC1
:1004E00011015E11016E110171110161110164119F
:1004F000015311015611013011286811014A1101EF
:100500002F11024D11015C110D5011035911FB0007
:10051000000009600148113711FE09603A11FE120E
:10052000C04811FE12C03C11FE12C03E11FE2580D3
:100530004011FE25804211FE44C04411FE06404693
:1005400011FB00010192114F120158122F001201EC
:100550000812010E12011512011C1201921101253F
:100560001201331201D511082C1201B41103C71165
:10057000024C120B431201A111033D12049E1107FC
:100580002C1201B41103C711024C120B431201A12A
:1005900011033D12049E11FB3100FE110900DA1116
:1005A000E611FE11E911EC11F211F511F811FB1130
:1005B000899108954198089507E800937A000FE320
:1005C00004B902E308B90CE307B903E00BB90AEF79
:1005D0000AB960D111F4299A01C06CD12A9A089500
:1005E000F89420E0E3E5F4E020832183009369029E
:1005F000789408955DD600916902EEE4F4E00C94DD
:10060000031748D111F4299A01C054D12A9800E067
:10061000E3E5F4E000830183FEC00091670200235C
:1006200019F132D109F43AD12DD128F033D111F496
:10063000299A01C03FD108D108F030D11DD128F04E
:1006400029D111F4299A01C035D1F8D008F026D16A
:1006500007D150F01FD111F4299A01C02BD100E02D
:10066000009367020E94C80E00916802002309F4FB
:10067000D2C00AD109F42A9A05D108F02A98E4D008
:1006800008F02A9AF9D008F02A98D8D008F02A9AC7
:10069000E7D008F4C0C02A9800E0009368020E94E6
:1006A000C80EB9C0E3D038F4F5D009F4B2C08CD587
:1006B00009F4299AAFC0E0D008F0A9CFEBD011F42B
:1006C000299AA8C0F7D0A6C0DFD019F4E3D079F7F3
:1006D000A0C0D8D008F09BCFDDD0A1F7F1CFC6D015
:1006E000A8F3CAD0C8F3BCD020F4D4D009F491C088
:1006F000DECF99D0389718F4CDD011F3E3CF93D053
:100700003A9798F390D03C97B8F38DD03E9768F322
:10071000A1D090F38DD008F07ACFEECFA7D028F3F8
:10072000ABD0F9CFA3D008F3FBCFA0D0C8F7B2D09D
:1007300011F4299A01C0BED02A986DC074D03A979E
:10074000D8F276D008F063CFF2CF9ED019F4289A71
:10075000419861C097D008F05ACF2898419A5BC061
:1007600085D018F289D0EECF8FD009F38BD020F24C
:100770006BD0E8F281D000F261D0C8F271D008F4F9
:10078000BBCF51D03F9798F265D008F4B5CF4BD08E
:10079000719768F248D0729708F4AECF44D073973F
:1007A00030F246D008F4A8CF3ED07E97B4CF6CD0BC
:1007B00009F49BCFDF0162D008F49ECF4BD008F440
:1007C00094CFA8CF61D009F490CF5CD008F494CF37
:1007D00053D008F48ACF44D008F48ECF24D03C976D
:1007E00028F458D0B1F0F0D4A9F46ACF1CD03E97C9
:1007F00030F450D009F464CFE7D461F40AC02AD0B1
:1008000080F311D0729708F002CF44D0A1F3DCD46A
:1008100009F429982A9AE3E5F4E00081118142D68F
:1008200000831183BAC6A3E5B4E0ED91FC9108956D
:10083000A3E5B4E0ED91FC9174970895A3E5B4E0CD
:10084000ED91FC9135970895A3E5B4E0ED91FC910D
:1008500033970895A3E5B4E0ED91FC917097089566
:10086000A3E5B4E0ED91FC9136970895A3E5B4E0DB
:10087000ED91FC9132970895A3E5B4E0ED91FC91E0
:1008800034970895DF01F4CFE3E5F4E000811181AE
:10089000012B0895009161020831089500916102D1
:1008A000083111F42998089500916102073109F483
:1008B000299A089500916102073109F42998089551
:1008C0004A92F6D42AD5FA93EA933A922A921A9245
:1008D0000A927A936A935A934A933A932A931A9371
:1008E0000A934FB6A895A6E4B2E0009169020530DC
:1008F00039F4FD0103891489D5D5038B148B04C009
:1009000000E0FD01038B048B81899289082F092B5C
:1009100009F00197818B928B87859089082F092B8D
:1009200011F001970FC000A1002361F4068D00FDB6
:10093000289A00FF2898078D00FD419A00FF4198F2
:1009400001E000A38787908B05A1002331F4038980
:1009500014890035134C08F45F9A07A5039507A77F
:1009600000A9039500AB0436B8F100E000AB05A583
:10097000039505A7009173024EE10E94631644237C
:1009800009F4C6D1009173020C3330F100E00093FA
:100990007302FD0106A5039506A706A50C33E0F03A
:1009A00000E006A704A5039504A70E943D1049F0A6
:1009B0000E943A1031F000917102002311F00E9460
:1009C000C00D00917202083139F400E00093720208
:1009D000FD0103A5039503A7009175024AE00E945B
:1009E0006316442349F5FD0185899689082F092B53
:1009F00071F001974AE050E08C010E94791641297C
:100A0000A9F4419B02C0419811C0419A0FC007A1AF
:100A1000013061F4068D00FD289A00FF2898078DAB
:100A200000FD419A00FF419800E007A3E6E4858BB2
:100A3000968B00E007A7DEDD4FBE24D05991699167
:100A400079910990199029903990E991F9917CD484
:100A5000A4D5499018957DD06ED020918400309116
:100A60008500169507956CD002E006BB00916F00DB
:100A7000026000936F00E89800E00093C5024FBF4A
:100A800001D01895099119912991399149910895A9
:100A90001A930A931FB75F995F980091520400233D
:100AA00009F00A95009352041FBF099119911895F6
:100AB0004ED00091C5021091C902202F002331F0C1
:100AC000215048F1285058F0A1F025C04A9902C0A1
:100AD000039521C011E01CBBE89A27D01CC04A9B9B
:100AE00002C020E801C020E01695122B1093C90225
:100AF000EFCF4A9B0BC02091C702F0E0E22FE05BF2
:100B0000FC4F108323952F772093C70203950DD0B8
:100B100011E01CBBE89A0093C5020DD0209188001B
:100B2000309189000DD053D0189510916F001D7F22
:100B300010936F0008950091C2021091C3020895AE
:100B4000200F311F30938900209388000895FA9375
:100B5000EA934A933A932A931A930A934FB70895C4
:100B6000F6DFD3D00481102F002341F0115008F19B
:100B7000175038F081F01A9581F01BC01281F29A5B
:100B800001C0108510FB16F45C9A01C05C981695A4
:100B9000108703950EC05C9AFCCFF29B08C0F19AB7
:100BA00010916F001B7F10936F00039502C05C983B
:100BB00000E004830081118120918A0030918B0034
:100BC000200F311F30938B0020938A00ACCF4FBF92
:100BD00009911991299139914991E991F9910895D2
:100BE0006FB7F894F19B1BC090D0208131815C9845
:100BF0004091840050918500420F531F50938B0009
:100C000040938A0014E016BB10916F00146010939B
:100C10006F0010E014830283F298F19807C0789473
:100C2000F29BFECFF8940093C402F2986FBF089530
:100C30001FB7F8940091C7020093C8021FBF089520
:100C4000FA93EA932A931A930A931FB700915004D8
:100C50002091C600F0E0E02FE053FC4F2083039585
:100C60000F77009350041FBF099119912991E991C1
:100C7000F99118955D9818950FEF1FEF2CE2015030
:100C800010402040E1F700C0000008950FEF1FE77B
:100C900024E0015010402040E1F700C0000008951A
:100CA0000EEF1FE801501040E9F70000089500E73B
:100CB00011E001501040E9F7000008950FE807BD6A
:100CC00002E004BD05E005BD00916E0002600093E6
:100CD0006E000895A80170D27BD221EE30E00E9410
:100CE000381013D00083118301E000938100F29A41
:100CF000F19A02E00093690001E00CBBE89A0091D0
:100D00006F00016000936F000895E2ECF2E0089537
:100D10005FD223E036EC30937C0030917C0030626F
:100D200030937C0030917A00306430937A003091B7
:100D30007A0036FDFCCF4091790050E0040F151F7A
:100D40002A9541F743E00E94791600936A020895BC
:100D50006097102EEFE6F0E08E0140E150E00E9437
:100D6000481700E0FE01E00FF41F1081111621F07A
:100D700003950031B8F300E060960895F999FECF2D
:100D800012BD01BDF89A00B50895F999FECF12BDC4
:100D900001BD20BDFA9AF99A08954AD0D801C90137
:100DA0003A01442406C02FEF82010A0F1B1F10D006
:100DB000439455244816590640F4F301E40DF51DFB
:100DC0000081002381F3202FEFCFE8E00C946C1713
:100DD000DCCF0E945D172801842F252FF9DF282FF3
:100DE00005D08201F5DFE6E00C946E1701E0400EBD
:100DF00000E0501E08951CD02801C901DA016624C4
:100E000006C0102FFD01E60DF71D108363947724B3
:100E10006816790640F48201060D171D29D00F3F90
:100E200081F710E0EFCFA80FB91F11977C92CDCFBB
:100E30000C945B171DD00F3F11F410E001C0102F70
:100E4000012F0895CAD3D80113D0802F11968D0198
:100E50000FD08F3F09F480E00F3F11F420E001C074
:100E6000202F182F022F282F220F220B322FDAC209
:100E700085CFA801F89404E6ADD6018B128B789447
:100E80000895F8946DD601891289012B789411F098
:100E90000C94E2120C944A1301E40093B800009100
:100EA000B8000A3018F40AE00093B8000091B900C5
:100EB0000C7F0093B900089544EA4093BC00409130
:100EC000BC0047FFFCCF46D0483021F00091B9006C
:100ED00010E09CC04EEA4093BB0044E84093BC0045
:100EE0004091BC0047FFFCCF35D0483119F032D0DB
:100EF000403411F71093BB0044E84093BC0040918C
:100F0000BC0047FFFCCF26D0483211F000E016C0ED
:100F100087D07ED007FFFDCF7ED0C1F72093BB00E6
:100F20006FD076D007FFFDCF76D081F704E969D086
:100F30006FD004FDFDCF04D003D001E010E0089590
:100F4000B6DEB5DEB4DEB3DEB2DEB1DEB0DEAFDE1D
:100F5000AEDEADCE4091B900487F089524EA2093DB
:100F6000BC002091BC0027FFFCCF46D0283009F000
:100F70002FC12EEA2093BB0024E82093BC002091CF
:100F8000BC0027FFFCCF38D0283141F71093BB00BD
:100F900024E82093BC002091BC0027FFFCCF2CD07C
:100FA000283231F73DD034D007FFFDCF34D001F7E0
:100FB00004EA27D02DD007FFFDCF26D00031C1F69F
:100FC0000FEA2ED025D007FFFDCF1ED0003481F6CA
:100FD00017D01ED007FFFDCF17D0083549F6009176
:100FE000BB0014E91093BC001091BC0014FDFCCFB1
:100FF000102F110F110B08952091B900287F08952B
:1010000004E80093BC0008950091B900087F08959A
:101010000091BC0008950091B900087F083208953E
:101020000093BB0004E8EDCF0E945717A6E4B2E09E
:1010300085E994E003EE10E01BDF093269F029E254
:1010400003EE0E94781220E009ED0E947812C2D0CF
:10105000F3D006D10E94C81445E554E058D5B8D065
:10106000CADEAC0154D58901C6DEAD0155D5B9D56E
:1010700046E852E02EE130E006E8B3D544EA52E01B
:101080002EE130E004EAADD54CE452E025E030E05A
:101090000FECA7D534D5A7D500937C020AED10E05C
:1010A000D1DE280139018BD036870CED9FD5802EFB
:1010B00000937D020DED9AD5B02E00937E020EEDC9
:1010C00095D5A02E00937F0200EE90D5902E12D5DC
:1010D00001EE8CD50BD502EE89D50093610204EEAA
:1010E00085D50E94C91405EE81D5009380020EEFCC
:1010F00004D5009383020FEF00D500938402009182
:101100009504002309F466D000914602002309F4F7
:1011100093D000914C02002309F4A2D0042D05299C
:101120000629072949F40E94681220E048D0268742
:1011300040E855E241D052D5882039F408E00093C8
:101140007D0228E00CED0E947812BB2039F40EE4F9
:1011500000937E022EE40DED0E947812AA2039F44D
:1011600001E000937F0221E00EED0E94781202E080
:10117000901608F4BED4009161020F3F21F024D0F4
:1011800051F088DB41F007E1009361022091610298
:1011900002EE0E947812009183020F3F19F400E0E2
:1011A00000938302009184020F3F19F400E0009342
:1011B0008402ECE00C94681760E070E00895FD0193
:1011C00003871487258708950091610207310895E8
:1011D00000E0B4CE09E30093950404E30093960481
:1011E0000EE20093970401E30093980403E3009355
:1011F000990407E300939A040EE200939B0401E331
:1012000000939C0409E300939D0403E300939E0470
:101210000EE200939F0402E30093A00401E3009315
:10122000A10408E30093A20400E00093A304AC012E
:1012300020E430E08901CDC405E30093460200E3D9
:101240000093470205E30093480200E3009349023C
:1012500000E000934A02AD0126E030E000E8B8C4A7
:1012600001E300934C0203E300934D0207E3009374
:101270004E0204E300934F0200E0009350024CE45E
:1012800052E025E030E00FECA3C43ED00EEF19EFA2
:1012900081D40330104018F49C010E94651254C0A0
:1012A00007D0D80101C0DDD10D910023E1F775C150
:1012B000BA93AA9308950E945D17D80129010E944C
:1012C000101305C0FD010191DF01CBD101968415FA
:1012D0009505C4F388CD19DD06811581101709F431
:1012E0000AC0102F13951F77168310E0F801E05BFA
:1012F000FC4F008108950FEF1FEF089505D001C046
:10130000B0D199D0E9F720C09A938A93C801089583
:1013100004D028ED2093C10004C09A938A930895C5
:10132000FCDFEEE4F3E000831183A80160E070E0ED
:1013300000E010E12EE030E00E94D816C8010197CD
:101340009093C5008093C40089919991089500936A
:10135000CB02055029F00A9531F00A9549F00DC0ED
:101360001AD00B7F07C017D00B7F13D0026004C0C8
:1013700012D004600ED00D7F24C00DD00460F5CFD4
:101380000093CC02023007D011F4086001C0077F3F
:1013900018C00093C2000091C20008950093CD02CE
:1013A000055419F00A5021F008C0F5DF006207C0AB
:1013B000F2DF0062EEDF006104C0EDDF0F7DE9DFE8
:1013C0000F7E0093C20008951091C00015FFFCCF5E
:1013D000F8940093C6005D9A52CDE0E5F4E00181F7
:1013E0001081101709F487CF102F13951F771183E1
:1013F00010E0F801E053FC4F7CCF8DD51123EAF3C8
:101400000895EBD0D80100E00C9305E07AD170D7B5
:1014100011F474D1E1F78D938F3F9F4FB1F702C064
:1014200010E0A096E4E00C9470176EDF01C00CD7BA
:1014300002D0E9F789CFFC010591CF0120C638DF42
:10144000D80101C001D70D910023E1F7A6C0F0DC5F
:101450002D01A02FC901BCDE390120E0E42DFB2FB6
:101460000083E42DFB2FE00FF11F20831BD00230FF
:101470001207B8F330DF11238AF00D30D9F30A30A8
:1014800081F0AA2349F0F201008300E011E0410E4F
:10149000501EF2010083AA953C01ECCF08DC41D537
:1014A00049F793CC0F5F1F4F089597D0C80100E014
:1014B000E82FF12F008305E024D11DD10FE1DC01DD
:1014C0000E94D213FC010081002311F417D1A9F767
:1014D00019D5A8CF0E94941205E013D152C019D09B
:1014E00000E0009364020093650208952898419AF1
:1014F00000E00093640201E0F6CF32D306A1013090
:1015000031F001E005D000E0068F01E00FD0089532
:1015100006A328984FC824D306A1002331F000E089
:10152000F7DF01E0068F00E001D00895078F08EE95
:1015300013E00787108B00E000A308958A93A0971B
:1015400080D6309911C00E9409130FE710E00E9465
:10155000CF1404E810E00E94CF1498DB5C988FE071
:101560000E9409138A95E1F7309907C00E94091378
:10157000429A5C980E9409134298C4D4A0960C9495
:10158000D80220E137E20FE1DE0161DF08810023AC
:1015900019F477DC0023A9F7A096A991B9910895D1
:1015A0001CD0A09780E00E9409130AE613E0E1D264
:1015B0000E940913A6D40EE613E00E940A13A3D0DA
:1015C0008395863008F0FCD293D069F78ED059F716
:1015D00002E713E0CED295D424CF0C945F170EE728
:1015E00013E0C7D205ED14E0E1D70EE713E08ED685
:1015F00005ED14E032D006E813E0BBD207EE14E0AC
:10160000D5D706E813E082D607EE14E026D00CE822
:1016100013E0AFD20CEF14E0C9D70CE813E076D694
:101620000CEF14E01AD001E913E0A3D200E412E0B9
:101630000E94BD1401E913E06AD601E412D001E46E
:1016400003D6B5D70BD05CD046DE0F3F1F4F11F04D
:101650000C944A1353D0C1F7B5C7F1DE04E813E088
:1016600055C6BECABADF6797C80108E092D300E941
:1016700010E04CD60CE910E07CD2009195040F3FAD
:1016800099F033D631D60EEA10E040D68C012CD634
:1016900000EB10E03BD629D60E94BD1403EB10E00E
:1016A00068D28C017FD702C008EB10E062D228D04C
:1016B0002AD01ED021F019D011F001E014C020D0A2
:1016C00002C00F34D1F317D00FE10E94D11316D00E
:1016D000A1F3098118811334A1F70F3471F708853C
:1016E000063459F300E067969DCE09810B340895C6
:1016F00008810F34089520E137E20895C2DBBFC4AA
:101700000CE310E0B6CB20E137E20FE1DE019FDE13
:101710000881002319F4B5DB0023A9F708950E947E
:1017200056172801F80100810E3031F501810E3085
:1017300019F502810E3001F50381A481B0E0EA0FB2
:10174000FB1FC58010E08824992408C0F201E80D31
:10175000F91D2581120F21E0820E9B1E8A169B0621
:10176000A8F326E4A22E22E0B22E11951C1539F022
:10177000F7D1018D128DFDD1EDE00C946717F0D1FA
:101780008789908DE2E8F4E00C940317A7D1E2EC8E
:10179000F4E00C94031700E619E0E2D1038715C0CA
:1017A00000EC12E1FACF94D6F8CF00E418E3F5CFBD
:1017B0001BE409C000E810E7F0CF16E904C000EC14
:1017C0001AEDEBCF11EECCD1B3871487B587B6876E
:1017D000F201768070927E02678060927D02408482
:1017E00040927F02BDD183859485A585B6858C0105
:1017F00097DD072D0E941116062D0E940F16042D4D
:101800000E940D16AC01BD01E9D1272D0DED70D65A
:10181000262D0CED6DD6242D0EED22C086D165D57A
:1018200080D118F488D1E4D101C05BD1C2D1B8F322
:101830006CD18901B2DA15C078D172D118F47BD19C
:10184000D7D101C04ED1B0D1C0F364D110E0F2CFF6
:1018500045D150D1002309F44CD12091810200EEF2
:1018600047D681D188CFF201258120937C0209EDF2
:10187000F7CF5BD155D120F468D126838CD102C03B
:10188000F801B6838CD1B0F301E030D106E0A00EB0
:10189000BB1EA50125E030E00FEC9AD121E027D650
:1018A0008FD166D17DDE68CF02E020D122E01FD645
:1018B0005FD186D161CF39D133D120F446D121AB6C
:1018C0006AD102C0F801B1AB6AD1B0F303E00ED126
:1018D00016D17ED123E00BD673D1C3CFFFD00093B6
:1018E0006E02BFCF22D104C0FCD063D108F0B9CFC3
:1018F000FCD417D1C8F71FD17BD1F7CF16D104C0C4
:10190000F0D052D108F0ADCF0BD1D0F714D170D1B7
:10191000F8CFE4D000937C02A4CFF7D000E461D1EB
:10192000F9D061D1F7CF6091840220918302D2D0A7
:101930000CE02BD21801068110E0200E311E422F40
:101940000CE00E947116060F151F201631060CF4CC
:101950000FCF478106E038D11581121B0CE0109F94
:101960000681000E061A09F00A940AEB009E002D6B
:1019700010E0005E114B800F911F0BD10196502E8D
:1019800000D10196500EFDD0500E6BDE8C018ADD29
:1019900001D1402E66DE51945418052D62DEECCE46
:1019A000F20125812093800205EE5ACFF89496D05B
:1019B00000936F0206810093700207810093710209
:1019C00000850093720201850093730202850093E3
:1019D00074027894D5D045CF7DD00AEBF5D04681FE
:1019E00006E0D3D140D320E08C0130E000521E4409
:1019F00020403040083F1A422040304008F0B8CE26
:101A000007E0802E9924F201E80DF91D208130E0D5
:101A10008C015AD50196BFD00DE080169B0698F335
:101A2000A2D0A7D0ADD0A8CEF20125812093830209
:101A300006810093840230E00EEF56D0209184029C
:101A400030E00FEF51D0C6CF58DD0BCF64DD09CFAA
:101A500046DD07CF4BDD05CF3DD00AE0BBD0058B7F
:101A6000168B01E007A3FDCE00916C02002319F054
:101A700006E913E080CE08E913E07DCEF2019581FE
:101A80000681802F9084818466247724278130E02A
:101A9000192F1AD5202F0196212B09F469CE292D53
:101AA00030E048D20196212B09F462CE282D62D075
:101AB00009F45ECEF201E60DF71D22855BD009F434
:101AC00057CE01E0600E7B1E00E160167B0690F3AE
:101AD0000C2D64CFF201458150E00895F20105819B
:101AE0000895F801B08308951CE7EEC400938202C4
:101AF000089505E00093810208951CE74BC047E775
:101B000052E025E030E004ED089545E954E020E49A
:101B100030E0089546E452E026E030E000E8089521
:101B20008501060D171D6A1649C005E0802E99240F
:101B3000662477240895F201E80DF91D20812A52C8
:101B40002631208108F0205D0895F201E80DF91D8D
:101B500020812A522631208108F0205DF801089565
:101B6000E6E4F2E00895E6E4F2E00789108D0895D6
:101B70008C01C4CB30E08C019FD901960C944804B1
:101B8000F9C10E94F0058C01E9D90196500E0E941E
:101B9000F0058C01E3C901E0800E9B1E089501E071
:101BA000600E7B1E05E009C001E0600E7B1E06E0B2
:101BB00004C001E0600E7B1E00E460167B06089501
:101BC00001E000936B02089510E00E9471169ECB15
:101BD00010E0E3C810E00E947116C2CF0AED10E0D9
:101BE000F8C810E008C910E006D909ED10E022C9D4
:101BF000F8012083D0CF0E9455172897CCD0CC2451
:101C000003E40A830CE40B830FE40C8303E50D83E8
:101C100005E40E8304E40F8304C004E00E9432163E
:101C2000BAD04091810250E00CE3AFD022D9A1D0CC
:101C300009F458C001E00093680203E0AAD035011E
:101C40005BD100E008830983442455240A2DA09227
:101C5000CE02FAD2FE013296DD24EC0DF41D008195
:101C60006016740411F4C39401C0CC2482D009F42A
:101C700053C000E840165D040CF04EC06A2C712E73
:101C80000A2DE2D201E0400E5D1CF201E253FD4F4D
:101C9000A082FE013296EC0DFD1D008160167D04D0
:101CA00011F4C3943EC0CC2403E460167D0409F40F
:101CB000C3940881198101311742C4F201E360160F
:101CC0007D0469F4452859F400916E02002339F02F
:101CD00000916102C6DC00916A02C3DC59D00EECAF
:101CE00012E01DDD4CD0A1F101E00093670202E09B
:101CF00050D0AA24BB24442455246092CE023FD065
:101D0000C9F000E8401600E05006A4F46FD8F201D4
:101D1000E253FD4F608212C008811981C3DB088342
:101D2000198305E0C01628F20091D1020D3109F2A5
:101D300000E01BC001E0A00E00E0B01E05E6A0160A
:101D400000E0B006E4F252D892010EEC12E0B3DAF1
:101D5000D5DC09F06CCF81309040A040B0400CF051
:101D60005CCF0AE913E0D2D201E02896EEE00C94B1
:101D70006617B1DA58010FEFA016B00608952DDBF3
:101D800038010FEF60167006089510E00C9471167C
:101D900009E010E073C780E090E0A0E0B0E00895B3
:101DA0000E9453172197C801D90144245524488221
:101DB000BB24AA24CC24DD24AED048010FEF80162A
:101DC000900609F479C0F601309669F0319769F010
:101DD000319769F0319769F0E150F04018F0E15126
:101DE000F04018F165C0482C63C0888261C0B82CEF
:101DF0005FC0582C0881A42CA00EAB0CA80C02E0EC
:101E0000501609F455C028819ED019F402E01CD266
:101E10006FC02B2D98D0D1F3282D95D0B9F374D065
:101E200008F446C02FEF83D043C076010DEFE00EDB
:101E30000FEFF01E71D00CF0A80C02E0501659F014
:101E4000042D0E151F053CF0940174D055D0212BA4
:101E500011F400E0DCCF10E0E414F10661F400E1DD
:101E6000401648F4552039F4602E77246418710A1E
:101E700065D057D0E9F750D0DCF4A19469D868D880
:101E800041D00A2D10E00815190511F42CD30DC00E
:101E900000E0DAD1042D10E00D5F1F4F212F220F3B
:101EA000220B801B910BA20BB20BCC24CA94DC2C0E
:101EB00001E0C00E00E0D01E01E0501609F07CCF1A
:101EC00004E0C01600E0D0060CF476CF1DD010F070
:101ED00020E02DD008D32C013D0108EC0E94F7062C
:101EE000601E701E2BD084159505A605B705D0F38E
:101EF0002196E0E10C9464178F5F9F4FAF4FBF4F67
:101F00000895C6D60C94180680300DE7900700E0BF
:101F1000A007B007089561CA042D10E00E151F0533
:101F200008950FEF600E701E062D0729089530E00A
:101F30001DE7CAC28C01A8D6202F08952FEF30E0EC
:101F40008C01A2D6D9CF30E08C019ED68F5F9F4FF7
:101F5000AF4FBF4F0C94480403DE11A505AD101B15
:101F60000CE0109F02A5000E06AD001A402D50E0B7
:101F70000AEB0BCF0E945A1780D009F456C07AD0D2
:101F800009F453C000918302002309F44EC000916C
:101F90008402002309F449C040907102DDDFC801CA
:101FA000A12FAA0FAA0BBA2F093B08E09007A04067
:101FB000B040D8F5E42DF0E0319748E150E08F01D2
:101FC0000E947116212F220F220B322F4091720294
:101FD000F3D8040F151F251F351F44E60E948D16E8
:101FE00042E00E94AD162801390144E641D0842E1A
:101FF00044E650E0E1D8820193013AD034D0C9DD03
:10200000802F22D100E0882099F414E0819F812D57
:1020100080FB0EF401E081FB4EF40260002321F00E
:102020000A95D1F00A95D1F068DA1AC00D7FF6CF83
:1020300019E1811629F482958F7080FB5EF3EBCF56
:1020400012E3811619F486958695F7CF1BE4811665
:1020500059F780FBFEF2DFCF5EDAE7CF40DAE5CF5B
:10206000E9E00C946B17800F911F805E914B0895EF
:102070000C94B5160091700202C000916F0200230B
:1020800008950E945717A0978FD019F406EA13E01D
:1020900002C000EC13E08DD082D309F482C084D05A
:1020A00019F40AED13E002C006EE13E082D0F894B2
:1020B00088859F81AA85B9854C845B8468887F84E4
:1020C0008A889988AC880B8910918002112309F5C0
:1020D0001AE0019F0A0C00EF000E00926F02919E21
:1020E000080C000E00927002719E060C000E009209
:1020F0007102519E040C000E00927202B19F0A0EF2
:10210000000E00927402919F080E000E009273025E
:102110003FC04DD0B02EB29400EFB0220A2D47D070
:10212000B02AB0926F02092D42D0902E929400EF07
:102130009022082D3CD0902A90927002072D37D023
:10214000702E729400EF7022062D31D0702A70929A
:102150007102052D2CD0502E529400EF5022042DE8
:1021600026D0502A509272020B2F21D0B02FB29558
:10217000B07F0A2F1CD0B02BB0937402092F17D058
:10218000902F9295907F082F12D0902B90937302EE
:1021900078940AD019F402EF13E002C000E014E0D2
:1021A00008D0A0960C94D9080091800268CF0C94B6
:1021B000A8063BD98E0125C90E945A17C801822E54
:1021C000732E2A01DB016624F801608206C008E054
:1021D0003BD000E239D008E037D00FD9102F18508B
:1021E00041F0155089F4AC019D0182010E94CD0699
:1021F00037CF00E229D0662081F36A9420E0FC0109
:10220000E60DF21F2083E7CF102F11521E35F8F68E
:1022100011E0711621F4102F10531A30C0F6262D3C
:1022200030E0E82DF0E031972E173F0784F6FC01EF
:10223000E60DF31F00836394FC01E60DF31F30836A
:10224000CBCF0CE001C00CE0BFC867D851D0F1F390
:102250000E9446068C01EAEDF4E00C94071774C85E
:10226000FCD425853685E0E1F5E00C940D1701E0FE
:10227000EBDFECCF02E0FCCF04E0FACF05E0F8CFD3
:1022800006E0F6CF07E0F4CF08E0F2CF09E0F0CFA8
:1022900003E0EECF00917D02EBCF00917F02E8CF0B
:1022A00000917E02E5CF00917C02E2CF0091810295
:1022B000DFCF00916102DCCF00E0DACF16D014D07E
:1022C000C5CF06E412E0FBCF0EE014E01FD0BECF76
:1022D0000CE412E0F4CF05E514E0F1CF06E812E0DB
:1022E000EECF04EA12E0EBCFAAC805E914E00895A6
:1022F00074D8C8010F3F0FEF900708950AE114E06A
:1023000006D000E214E002D002E214E08EC88DD8BC
:1023100000E412E0E9CF61D980E006E03ADDEEDFCB
:1023200005E0EFD9F8DDD801882319F4E7D909F4DD
:10233000B4C08D01E2E4F5E00C94071781E085DF7D
:10234000F1CFBDD0055471F0095011F00A9541F05C
:102350000EE400937E0220917E020DEDC9D0E2CF03
:102360000FE4F7CF05E4F5CFAAD0055329F00250CA
:1023700051F00A9551F009C005E000937D022091CB
:102380007D020CEDEBCF07E0F8CF08E0F6CF97D059
:10239000015311F00A9539F001E000937F0220917A
:1023A0007F020EEDDBCF02E0F8CF89D0E8E9F5E05F
:1023B0000C94031700E619E020E08DD025872687CE
:1023C000438554856585768509DCACCF00EC12E148
:1023D000F3CF00E418E3F0CF00E01BE47CD00587E6
:1023E0000687EECF00E810E7E7CF00E016E9F6CF6A
:1023F00000EC1AEDE1CF00E011EEF0CF69D0DCCFB8
:1024000060E470E040E06CD005E514E0D5DE8ACFF2
:1024100060E470E0AB019B0168DFF8CF6EE170E033
:1024200046E85ED006E812E0F1CF6EE170E044EAE3
:1024300057D004EA12E0EACF66E070E040E850E0EE
:1024400031E026E006E412E0E1CF39D0005388DB2A
:1024500006AB202F09ED82CF65E070E04FEC40D055
:102460000CE412E0D3CF2BD07BDB03AF023010F4AF
:1024700005E003AF23AD00EE71CF21D071DB038FF8
:10248000238D02EE6BCF23E030E01FD020E030E060
:102490000FEF19EF19D046CFF7980C94120A0E944B
:1024A000500621D000E01DE720E030E079DC3ACF93
:1024B0000E94500602E0C8DE0E94E808F5CF0E94A4
:1024C000FD090023E1F30895DFC30EEF19EFFCCF00
:1024D00000E815E20895E6E4F2E003871487089522
:1024E00050E09B01089501E0AFCE05E052CC01EE33
:1024F00010E00C94E806A5DE0BE214E007DF03D041
:1025000002D087D086C0C4D382C00ED00EEC10E0BB
:1025100081D05AD00CED10E0ABD00D85013311F411
:1025200000E001C04AD046C0BA93AA93A09708958C
:10253000FBDF01EE10E06ED047D00F81033581F54F
:102540000885093469F509850D3451F50A8500328D
:1025500039F50B85003521F50C85093409F50D8514
:102560000E34F1F40BEE10E004DB0CE412E01AD0B0
:1025700051D02AD004EF10E07BD00F81023571F4E6
:102580000885053459F40985013441F40A85043479
:1025900029F40B85093511F422D002C00ED001C0F8
:1025A00000E008C073D306EB10E008956FD304E891
:1025B00013E0DFCAA0960C94CD0A04E010E05ED3CD
:1025C0000E946A0A01E0089520E137E20FE1DE018E
:1025D00063D30881002319F455D30023A9F70C9481
:1025E0006A0A1BD002C017D065D013D009EF10E0E3
:1025F00011D052D014F001E008C00985013399F7D9
:1026000003E011E035D007D03AD00C94100A40D343
:102610003FD33EC33FD30EE174C80E945F17A0971B
:1026200080E090E00895F9DF02C0F5DF43D0F1DFEC
:1026300008E011E0EFDF30D014F001E008C00A85B7
:10264000013399F703E111E013D0E5DF18D00C94C2
:10265000100A0FE710E01ED320E137E20FE1DE01A0
:102660001BD320E137E20FE1DE0116D304E912E0CB
:1026700007D38E010E941F0A00EB10E047CE20E135
:1026800037E20FE1DE0108D30881002319F4FAD202
:102690000023A9F700E0089520E137E20FE1DE0111
:1026A000FBD20881002319F4EDD20023A9F786306C
:1026B00000E022CE20E137E20FE1DE01EDD2088119
:1026C000002319F4DFD20023A9F70196A2CF0E94BC
:1026D000ED0A2A97A5DF16DC04E314E064D0CCD21F
:1026E000C9D204E1A7EEB4E05DD00091E704002375
:1026F00011F4BED2A9F70091E704002311F401E020
:102700004BC005E1E5EDF4E0E00FF81F1289163447
:1027100009F4828B0A950031A8F7F3DB0EE314E08D
:1027200042D0AAD2A7D201E1A5EDB4E03BD00091FE
:10273000D504002311F49CD2A9F70091D5040023FD
:10274000F1F2DFDB06E414E014DA0AE095D292D26B
:102750000AE027D024D011F48BD2C9F720D079F227
:10276000FE0110E0E80FF11F0081003281F406C085
:10277000E5EDF4E0E90FF11F27A393958395FE01A2
:10278000E80FF11F2081222399F32C3289F78395DA
:102790008A3030F3B6DB00E02A960C94120A0881E6
:1027A0006ECCDE0179C276D220E137E202E0DE01B2
:1027B00073D20AE0089520E003C02395203438F452
:1027C000F0E0E22FEB56FB4F0081002309F462CFCB
:1027D0000E3299F300530A3080F3F4CEA5DE31DDDA
:1027E00000915504002309F08DC009E111E0D7D014
:1027F0000C850D3409F043C00D85043509F058C02F
:102800000E85033509F07EC001E0C3D003E211E07C
:10281000C6D001E311E0ADD900918502002351F04B
:102820000A9509F47BC00A9509F47EC00A9509F45B
:1028300081C086C00EE311E069DD03E511E099D99E
:1028400005E514E09BD006E812E098D004EA12E017
:1028500094D003E511E08DD906EB10E0A0D004E0A0
:1028600012E09DD000E112E09AD00DE112E097D085
:10287000A2DF013009F068C002E312E067C006344D
:1028800051F50D850136F1F50E850237D9F50F8525
:102890000032C1F508890534A9F50989013691F599
:1028A0000A89033779F50B89043761F503E0ADCF69
:1028B000053641F50E85073629F50F85013611F5E8
:1028C00008890634F9F409890F36E1F40A890E36CD
:1028D000C9F402E09ACF0234A9F40D85013469F4F9
:1028E0000E85093479F40F850B3461F408890134BD
:1028F00049F409890C3431F4D9CF073519F40E8520
:102900000334A1F200918502002309F07FCF0091EA
:102910005504002309F47ACF01E02DC005E511E04C
:10292000F5DC07E611E097CF05E811E0EFDC0BE9F5
:1029300011E091CF06EB11E0E9DC02ED11E08BCF65
:102940000CEE11E0E3DCE8CF00E412E028D00EE466
:1029500012E025D00BE512E022D000E0088305E666
:1029600012E058DE0E94830B01E712E081DE37DEC1
:1029700016DF91F200E010E01DCE88C187D103E59B
:1029800011E088D10EEA10E085D103E511E0F1C82D
:1029900000E000938502089579D100EC12E07AD12D
:1029A0008E010C94550AA097A89544240E94E8082B
:1029B000F1D90E94DC020E944C070E94140801E039
:1029C00000936202009363024092640200936502E6
:1029D000209A399A0E94890AA89544D100E717E104
:1029E000BFD80787108BA89573DD0E946A0600E0A8
:1029F00011EE0E9488090EE414D108E010D101E024
:102A00000CD10E945E067894F79A85DC26D10E944C
:102A1000900900917E0205D100917D0200D10091C4
:102A20007F02FBD062DDF3DDA0E02BDB26DB41F093
:102A300021DB31F000917102002311F0A1D804C014
:102A40000A2FA395023088F356DD06C004E0A1D911
:102A500009E912E05BDCDBDD48DD0E949E0AD9DD7E
:102A6000D8DDEFDB05E712E051DCD3DD439AD1DDA1
:102A700043985C9ACCDD0EE712E0DCD003E812E06C
:102A8000E4D0C7DD08E812E0D5D00EE812E0DDD0D2
:102A9000E0DD0881033469F409810136F1F60A8129
:102AA0000C36D9F60B810C36C1F60D810235A9F62C
:102AB000D0DD0E94780B89F60E94750B71F6B0E0AC
:102AC0008EDD23DD002311F633DD002329F004E041
:102AD00060D904EA12E0BECF00918202013029F4ED
:102AE0000FEA12E0A3D058DF20C0023019F403EC43
:102AF00012E0F8CF0330D9F404ED12E097D03DDFB7
:102B000003EE12E036D807E712E046DF0E94780BAA
:102B100061F40E94750B49F4A0E022D8EA0FFB1F74
:102B200001A90683A395A530C0F3B093820257DDB7
:102B300058DD012B29F002E198D007EE12E08ACF90
:102B40004EDD71DD012B29F003E18FD003EF12E0A0
:102B500081CF02E087D043DDBADD002329F004E114
:102B600018D900E013E076CFA091E3041091E204BD
:102B70000AE0109FA00DA051A53610F0A4E603C0F6
:102B8000AF3008F4AFE02BDDBB2341F427DE012B8F
:102B900029F0FEDE20E004EEABDC5ECFB1E01FDD0D
:102BA00006E412E00E94320B502E002329F50E9409
:102BB000EF0A002309F5ECD80AE013E0A7DB442470
:102BC0002091850204EE94DC16D8002300E110E089
:102BD00011F0E0D841CFDED80AE113E024D04394CD
:102BE00001E1D7D855245A1608F0B5CF12DD03E617
:102BF00013E08CDB5394F7CF00E1CBD843945520FE
:102C000021F40EE213E00FD003C006E413E07EDBF4
:102C100003E0401628F344241FCF0C94C0090C9401
:102C2000A7090C94CE092CD00C94D00A33D00CE414
:102C300012E008952FD020E137E20FE1DE012CD021
:102C400020E137E20FE1DE01ADCD1AD08E010E9406
:102C50001F0A00EB10E014D0DCCCE6E4F2E00385C0
:102C60001485089510E00C94450910E007D0EBCAD4
:102C70000C947E0B0C947B0B0C94810B0C94F00247
:102C80000C94150A0C9441070C945C070C945009A1
:102C90000C943C060C947E090C94270A000088953D
:102CA000FECF0FE30DBF02E00EBFC0E0D2E00E94F6
:102CB0007917002311F00E9489170E94D3140E94F3
:102CC0004E160C944E160024E8E0EA9532F0001FF0
:102CD000001C0416D0F3041AF8CF001F402D0095F5
:102CE0000895149F102D059F100D049F002D110DA8
:102CF000089500241124EFE0001F111F001C111C77
:102D00000416150610F0041A150AEA95AAF7001F12
:102D1000111FA0010095109508952224349F302D95
:102D2000259F300D169F300D079F300D249F202DBD
:102D3000310D159F200D311D069F200D311D149F53
:102D4000102D210D321D059F100D211D321D049FD8
:102D5000002D110D221D321D08954A952AF0369539
:102D6000279517950795F9CF089500241124100190
:102D7000E0E2EA9592F0001F111F221F331F001C92
:102D8000111C221C331C041615062606370688F370
:102D9000041A150A260A370AECCF001F111F221F3A
:102DA000331FA001B101009510952095309508952D
:102DB000FF27772312F4F16015D0332312F4F09536
:102DC00009D00E94B516F69508F404D0F69508F4DB
:102DD00009C0089530952095109501951F4F2F4FEC
:102DE0003F4F089570956095509541955F4F6F4F97
:102DF0007F4F08957591659155914591159011FA00
:102E0000259035900895F9DF041B10E003C0F4DF2E
:102E1000041B150B20E030E005C0ECDF041B150B94
:102E2000260B370BB8F010FC17C045910590E00F4A
:102E3000F11F0417100540E02407340758F436F456
:102E400004910024F101E01BF0090994E00FF11F47
:102E500025903590F101099411F4D6F7F1CF319610
:102E60000EF0319650E060E070E045914B3F48F045
:102E700089F34F3F29F04E3F11F0759165915591BF
:102E80004591041B150B260B370B39F318F3E7CFCD
:102E9000AF93BF93D80105900D9241505040D9F7A0
:102EA000BF91AF910895FA92EA92DA92CA92BA92D9
:102EB000AA929A928A927A926A925A924A92BA9371
:102EC000AA939A938A930895FF84EE84DD84CC8438
:102ED000BB84AA84998488847F806E805D804C80C6
:102EE000BB81AA8199818881F0E0EC0FFD1FEF0181
:102EF000089501E0089520E006D0E9F708952591AE
:102F000002D0E9F708952D9301501040202F212B76
:102F1000089586E49FE2FC0105911491FC0132962C
:102F2000A591B491FC01349625913491422F432B05
:102F300019F0F901E4DF01C0DEDF06961FE28235F9
:102F4000910748F308958E004002522F3102CE02BD
:102F50000000312E312E3100000000000000000082
:102F60000000000000000070170000000000006872
:102F7000006B0000010100010000000000000100E2
:102F80000100000000000000000000000000000040
:102F90000000000000000000000000000000000031
:102FA0000000000000000000000000000000000021
:102FB0000000000000000000000000000000000011
:102FC0000000000000000000000000000000000001
:102FD00000000000000000FFFF0000000008014E9C
:00000001FF
:00000001FF
